:020000020000FC
:100000000C9434000C94E90A0C94E90A0C94E90A63
:100010000C94E90A0C94E90A0C94E90A0C94250A58
:100020000C94E90A0C94E90A0C94E90A0C94E90A84
:100030000C94E90A0C94E90A0C94E90A0C94E90A74
:100040000C94E90A0C94E90A0C94E90A0C94E90A64
:100050000C94E90A0C94E90A0C94E90A0C94E90A54
:100060000C94E90A0C94E90A0FEF0DBF04E00EBFEF
:1000700046D57894C2D16FEF91D1DDD1FACFE39517
:10008000C8953196002009F0089500E00093B90466
:100090005FC5E4EDF5E1F4DF091679F4F1DF081648
:1000A00069F4EEDF071659F43196C895002D3196A4
:1000B000C895F02DE02F0995089531963196339625
:1000C000EACF90EF80EF21E008813CD1513011F46C
:1000D0001AD0F7CF702F17D00D3091F0352E088140
:1000E00031D10D3069F0351639F4982F872F702FE4
:1000F0000AD02395233099F7088124D1351609F0C9
:10010000089501D0F9CFDD1539F4CC1529F404E0B8
:100110000093B9041DC508952197089520E25ED18A
:1001200020E25CD120E25AD120E258D1392F4FD1C0
:1001300020E254D1382F4BD120E250D1372F47D174
:1001400020E24CD1089520E249D120E247D13E2F50
:100150003ED120E243D108950BE00093B904F8C4E6
:10016000D4E0CFE3552444247727BF7D0881CA9586
:1001700043940D3041F0E6D0523039F0B062513046
:10018000A9F35394F3CF052D0895B5FF7395EECFE2
:1001900004E00093B904DCC402E00093B904D8C4BD
:1001A0009F708F707F70EDD10895D4E0CFE3E03081
:1001B00099F308810083319721970D30C1F7AE2E56
:1001C000BF2E0895CDDF743038F60B2D033021F4A7
:1001D0000A2D043F09F452C0D4E0CFE377278827E3
:1001E0009927CC15AAF20881ADD0523029F4982F66
:1001F000872F702F2197F5CFD3DF672EFB2DEA2DA8
:10020000B77FBF7E99278827772777243196F330E9
:1002100011F4E53F59F0008195D0543039F0523057
:1002200089F77394782F892F902FF0CF072D033003
:1002300029F07394782F892F90E0F8CFB4FD02C095
:10024000B061E0CFADDF671699F118F4B8609F2E6A
:100250008E2EF33021F4E53F11F4B3FF0FC0B3FF4E
:1002600008C0761508F443C0F33019F4E53F09F4EB
:100270003EC0F33039F6E53F29F6089571DF0030CE
:1002800009F40895D4E0CFE3FB2DEA2DF13019F401
:10029000E03009F409C008810083319721970D30BF
:1002A000A9F7AE2EBF2E089502E00093B90450C402
:1002B0003197DF2FCE2FD13019F4C03009F468CF39
:1002C000088121970D30B9F70E2F0C1BA00E08F4F2
:1002D000B394D13011F4C03029F008810083219704
:1002E0003197F7CF3DDF003009F06CCF089538DF4C
:1002F000003039F10B2D013021F40A2D0050041586
:1003000098F2FB2DEA2DDF2FCE2FC419D0400C2FF1
:10031000A02E0D2FB02EF91519F4E81509F405C01B
:100320000081088321963196F6CFD4E0CFE3F92DF2
:10033000E82D3197088100830D3019F0319721970E
:10034000F9CF08955527102F1D3009F416C01F75D9
:10035000103009F402C01C3011F451E0089510313E
:100360000AF408951B350AF00895103412F053E092
:1003700008951A310AF452E0089554E00895CF33F5
:1003800019F427E02BD00EC028E03CD020E23AD070
:10039000212F38D0C3951DE0188304C02EE31ED052
:1003A000D4E0CFE334D0183051F31F3741F31A3083
:1003B00009F4F8CF18831D3049F0C03019F427E054
:1003C0000DD0F0CFCA95212F1DD0ECCF0895BED00F
:1003D000242F04D0232F02D00895202F0090C00096
:1003E00005FEFCCF75D3B6FF05C00090C00007FE28
:1003F000FCCFBF7B2093C60008952DE0EFDF2AE0FD
:10040000EDDF08952D3011F4F8DF0895E7CF8895DA
:1004100000000091C00007FFFACF1091C6000895B8
:10042000C895002021F0202DD9DF3196F9CF08950D
:10043000F7DFE3DF0895D4E0CFE30FEFC02E04E051
:10044000D02E08817FDF523009F4BCCED6DFA16008
:1004500001C0AE7F3DB73F3C20F408E00093B904F3
:1004600077C32FDE7D30C9F07B33B9F0032D023026
:1004700031F49F708F707F7084D022D0EBCF9F7546
:100480008F757F75213029F4032D033011F407D0C7
:10049000E1CFFFDD7D3009F00895A160089571542A
:1004A0007A3122F005E00093B90452C3705CA0FFDA
:1004B00011F406D00895F4E0E72F708101D008957B
:1004C000F3E0E62F70836A95633F20F406E0009323
:1004D000B9043EC308956395603022F007E00093AD
:1004E000B90436C3F3E0E62F70810895F4DF07E026
:1004F00007174AF001E0703019F0000F7A95FBCF32
:10050000702FDEDF08950AE00093B90421D3903004
:1005100039F0905D292F62DF803011F420E35EDF37
:10052000803019F0805D282F59DF705D272F56DF4E
:10053000089599278827745610F09395FCCF7C591D
:100540007A5010F08395FCCF765F0895432F46953F
:10055000469546954695405D4A3308F0495F3F70A1
:10056000305D3A3308F0395F089546FD475F4F70BC
:1005700036FD375F3F70440F440F440F440F342B58
:1005800008959330B2F4923032F0863092F4853090
:1005900012F0763072F4882321F00AE0700F8A9509
:1005A00081F7992309F4089504E68894700F9A95C9
:1005B000C0F701E00093B904CBC2EAEAF8E138DF02
:1005C00008951BDFF3E0E4EFFB1511F4EA1521F0C9
:1005D000208118DF3197F8CF10DF0FDFEAEBFBE166
:1005E0001FDF7A2D9B2D705091406ADF792FA1DF9C
:1005F0008EDFE8ECFBE114DF6EDF9BDF88DFFDDEE2
:100600000895AE7F27DF67DF94DF81DFF6DE089590
:1006100020DF24E2E3DE5FDF372FD9DEEEDE089550
:10062000AE7F18DF58DF072F56DFF4E0E72F008397
:100630000895A2FF72C0AE7F0DDF4DDF672E4BDF46
:10064000872F49DF772EF4E0E72F8083A062A86030
:10065000AA7F0895F4E0E72D0081061519F00395AF
:100660000083A0610895F5DE36DF072F34DF7017B1
:1006700019F0772725DF08957FEF22DF0895E9DE5F
:1006800070E000B605FE71E01BDF0895E2DE23DFB7
:10069000E72FF0E0708114DF0895DBDE1CDF072F09
:1006A0001ADFF0E0E02F70830895D3DE14DF072F08
:1006B00012DF709F1120F09B19F4702D01DF089557
:1006C0000FE00093B90444D2C4DE05DF7723F09B2A
:1006D00099F0072F00DF872F991B79E0881F7A9503
:1006E00041F0991F901B18F4900F8894F7CF08944D
:1006F000F5CF782FE5DE089501E10093B90428D203
:10070000A8DEE9DE072FE7DE700FF09B10F0D8DEE1
:1007100008950FE00093B9041BD29BDEDCDE072FA7
:10072000DADE701BF09B13F0CBDE089500E100933E
:10073000B9040ED28EDECFDE072FCDDE7023C0DEF1
:10074000089587DEC8DE7695BBDE089582DEC3DEBF
:10075000770FB6DE08957DDEBEDE072FBCDE702B80
:10076000AFDE089576DEB7DE072FB5DE7027A8DE90
:1007700008956FDEB0DE7095A3DE08956ADEABDE0D
:1007800071959EDE089571E09BDE089562DEA3DE22
:10079000072FA1DE701705C05CDE9DDE072F9BDEF4
:1007A000071770E082F779F38BDE089552DE93DE4F
:1007B000772309F0A26008950DB70E5F0DBF08956D
:1007C000A460089546DE0895B260089548819BDCD8
:1007D0003881CBDE732F74DE96DC3BDE089539DE84
:1007E0007ADECF93DF93D4E6C9EFCA950000E9F72C
:1007F000DA950000C9F77A95B1F7DF91CF910895A6
:1008000077275EDE26DE67DE01E007172AF0F09824
:1008100070FD01C0F09A08950CE00093B90498D1DE
:1008200018DE59DE472FF3E0E4EF0AC0FB1511F4A0
:10083000AE16E8F400810D3011F03197F7CF319703
:10084000772788279927FB1511F4AE1680F40081CD
:1008500079DD523029F4982F872F702F3197F3CFFD
:100860009F708F707F708DDE471701F7089509E044
:100870000093B9046DC1D4DFDF2FCE2F0895D0DFF0
:10088000A06C0895B2FF02C0B1600895B2600895EF
:10089000E0DD21DE272FA2DD08958895000000917C
:1008A000C00007FFFACF7091C600733009F4B26040
:1008B00007DE0895CEDD0FDE08E020E3771F08F4A1
:1008C00021E38CDD0A95C9F798DD089504EB70915A
:1008D000BA04779508F470277093BA04F1DD08958F
:1008E000427265616B200A0D0000D3E0C4EF6FEF28
:1008F000A160EED0A5FF03C08C2E9D2EAF7DA4FF7E
:1009000003C0D92DC82DAF7EA6FF03C04C2E5D2E8F
:10091000AF7BA7FF04C0DF2FCE2FB460AF77B0FF4F
:1009200003C0D52DC42DBA7FB1FF04C0CDD0DB2DBF
:10093000CA2DBD7FDB1511F4AC1678F4088102DDF9
:10094000A1FF04C0543011F02197D1CFAD7F5230B8
:1009500011F42197CCCF7EDDCACF089503E0B02EED
:1009600004EFA02EFB2DEA2D6FEFA0E0B0E0F1E048
:10097000E0E000E00193F330E8F3E43FD9F7F4E07E
:10098000E0E400E00193F430E8F3EA35D9F735DD2F
:10099000E2E2F8E14DDD0895E6EAFAE141DDE2E860
:1009A000FBE13EDD08E1202EF3E0E4EF3F2F0FDD19
:1009B0003E2F0DDD2AE312DD20E210DDF13011F4CF
:1009C000E03099F0308103DD20E208DD31972A9490
:1009D00059F413DD3F2FFBDC3E2FF9DC2AE3FEDC6C
:1009E00020E2FCDC08E1202EE9CF07DD06DDEEE9A0
:1009F000FBE116DD3B2DEBDC3A2DE9DCFEDCE6EA23
:100A0000FAE10EDDFADC0895E6EAFAE109DDEEE04E
:100A1000FBE106DD08E1202EF1E0EFEF3F2FD7DC10
:100A20003E2FD5DC2AE3DADC20E2D8DC0F93E0307D
:100A300000E0F0070F91B1F0F2BDE1BDF89A30B5DA
:100A4000C6DC20E2CBDC31972A9459F4D6DC3F2F68
:100A5000BEDC3E2FBCDC2AE3C1DC20E2BFDC08E1C7
:100A6000202EE4CFCADCE6EAFAE1DADCC6DC08953F
:100A7000E6EAFAE1D5DCE8EFFAE1D2DC08E1202E83
:100A8000E0E4F4E03F2FA3DC3E2FA1DC2AE3A6DC68
:100A900020E2A4DCEA3591F0319199DC20E29EDC81
:100AA0002A9459F4AADC3F2F92DC3E2F90DC2AE3F3
:100AB00095DC20E293DC08E1202EECCF9EDCE6EA18
:100AC000FAE1AEDC9ADC0895E0EEF8E0A9DC0895E6
:100AD0000090C00007FE0BC00091C600033111F466
:100AE000B06405C00091C600033009F4B2600895F7
:100AF000DF93D2E0DA950000E9F7DF91089506E28E
:100B000004B900E005B900E007B900E008B902E265
:100B10000AB900E00BB900270093BB040EBB74EBCD
:100B20000091000107270093BA0400E00093C5007C
:100B30000FE10093C40008E90093C10001E003BF86
:100B40000E94AE04489902C0D6D3CFDE36DD0895A8
:100B500054DC0091B904EFEAF5E0E00F099415C008
:100B600017C019C01BC01DC01FC021C023C025C095
:100B700027C029C02BC02DC02FC031C033C035C005
:100B800037C039C03BC03DC03FC0E2EDFBE13FD0C4
:100B9000EAEFFBE13CD0E8E3FCE139D0EAE5FCE137
:100BA00036D0ECE9FCE133D0ECECFCE130D0E0E015
:100BB000FDE12DD0E2E4FDE12AD0E2EAFDE127D01B
:100BC000E2E0FEE124D0EAE3FEE121D0E2E7FEE14B
:100BD0001ED0E6EAFEE11BD0EEEDFEE118D0E6E124
:100BE000FFE115D0E0E4FFE112D0EEE5FFE10FD028
:100BF000EEE7FFE10CD0E8E9FFE109D0EAEBFFE125
:100C000006D0E0EEFFE103D0E6E0F0E200D008DC41
:100C10000FEF0DBF04E00EBF0FEF0DBF6FEFA0E0B1
:100C2000B0E0EBDB26CA009164000F77009364000C
:100C3000772746DC0EDC4FDC01E00717A2F004E06A
:100C400070FD0AE20093B800459A449A0027009389
:100C5000B90000950093BB0004E00093BC0004E9D8
:100C60000093BC0008950CE00093B90471DF00917B
:100C7000BC0002FF25C0EDDB2EDC7093BB0005E855
:100C80000093BC000091BC0007FFFCCF0091B900AD
:100C9000087F083111F0003439F47091B90076956D
:100CA000769576950DDC0895003231F0083421F008
:100CB00002E10093B9044CDF04E10093B90448DF7A
:100CC00003E10093B90444DF0091BC0002FF21C09E
:100CD000C0DB01DC7093BB0005E80093BC00009111
:100CE000BC0007FFFCCF0091B900087F083239F43F
:100CF0007091B900769576957695E2DB089500338C
:100D000021F002E10093B90423DF04E10093B90468
:100D10001FDF03E10093B9041BDF0091BC0002FF59
:100D200023C071E0CDDB95DBD6DB01E0071702F1D4
:100D300004EC70FF04E80093BC000091BC0007FFC6
:100D4000FCCF0091B900087F003521F47091BB0001
:100D5000B7DB0895003521F002E10093B904F8DE15
:100D600004E10093B904F4DE03E10093B904F0DE7A
:100D70000CE00093B904ECDE0091BC0002FF11C04E
:100D800004EA0093BC000091BC0007FFFCCF009177
:100D9000B900087F083009F4089502E10093B9040E
:100DA000D7DE03E10093B904D3DE0091BC0002FF5B
:100DB0000BC004E90093BC000FEF0093BB00089543
:100DC00002E10093B904C4DE03E10093B904C0DE7C
:100DD0000091BC0002FF11C00091BC0004FF02C0E2
:100DE00070E809C00091BC0007FFFCCF7091B9000A
:100DF00076957695769564DB089503E10093B904C2
:100E0000A7DE009164000B7F0093640072E058DB62
:100E100020DB61DB03E0071742F0770F770F51D03B
:100E20000CB5037F072B0CBD08950DE00093B904AA
:100E30008FDE0FDB50DB01E007174AF00CB50062D4
:100E40000CBD70FD03C00CB50F7D0CBD08950CE00A
:100E50000093B9047DDEFDDA3EDB07E007177AF088
:100E6000072E73700CB5087F072B0CBD0DB5016004
:100E70000DBD02FC03C00DB50E7F0DBD08950AE047
:100E80000093B90465DEE5DA26DB2A98000000004D
:100E90007EBD0DB407FEFDCF7EB508952A980000F3
:100EA00000007EBD0DB407FEFDCF7EB509DB0895C1
:100EB00071E006DBCEDA0FDB2A9A70FD01C02A98BA
:100EC000089504B10C6204B905B1046005B901E5E7
:100ED0000CBD0DB50E7F0DBD0895009164000E7F11
:100EE0000093640000E000937B007727E9DAB1DA31
:100EF000F2DA00917C00007F7F70072B00937C006A
:100F000006EC00937A0000917A0006FDFCCF06EC17
:100F100000937A0000917A0006FDFCCF7091790071
:100F2000CFDA08957727CCDA94DAD5DA01E007171B
:100F300052F000917C000F73006270FD01C0006CE4
:100F400000937C0008950CE00093B90401DE74B1B5
:100F5000B7DA08957EDACADABEDA05B1072B05B929
:100F6000089577DAC3DAB7DA709505B1072305B9C2
:100F700008956FDABBDAAFDA04B1072B04B908952C
:100F800068DAB4DAA8DA709504B1072304B90895D1
:100F900060DAACDAA0DA03B1072370E0002309F4C9
:100FA00071E08EDA089555DA96DA75B9089551DA56
:100FB00092DA74B9089573B183DA089577B180DA5B
:100FC000089547DA93DA87DA08B1072B08B908954C
:100FD00040DA8CDA80DA709508B1072308B90895F1
:100FE00038DA84DA78DA07B1072B07B9089531DAED
:100FF0007DDA71DA709507B1072307B9089529DA08
:1010000075DA69DA06B1072370E0002309F471E0AC
:1010100057DA08951EDA5FDA78B908951ADA5BDADA
:1010200077B9089576B14CDA08957AB149DA08951E
:1010300010DA51DA7AB908950CDA58DA4CDA0BB1D1
:10104000072B0BB9089505DA51DA45DA70950BB123
:1010500007230BB90895FDD949DA3DDA0AB1072B08
:101060000AB90895F6D942DA36DA70950AB107233B
:101070000AB90895EED93ADA2EDA09B1072370E0F9
:10108000002309F471E01CDA0895E3D924DA7BB96E
:10109000089579B115DA0895DCD901E8009380004C
:1010A00009E000938100002700938200219A13DA5F
:1010B000002700938900709388000895CAD903E837
:1010C0000093800009E000938100002700938200D4
:1010D000219A01DA072FFFD97093890000938800C5
:1010E000089500270093800008957727E9D9B1D9A2
:1010F000F2D907E0071772F00091BB04087F702B4C
:101100007093BB040027009382000093800000933B
:10111000810008950AE00093B9041ADD71E0D0D986
:1011200098D9D9D901E007174AF00091BB040F778D
:1011300070FF01C000680093BB0408950CE00093A9
:10114000B90406DDCF93DF938827772776BB80939A
:10115000850070938400B09A0091BB04902F907822
:10116000C894991F991F96600770E9EBF8E0E00FAB
:1011700009947AC006C005C004C02AC029C028C08E
:101180004FC0033008F005E0909381008093850004
:1011900070938400DAE0C3EFCA95000000000000FD
:1011A0000000D1F7CFEFCA95000000000000D9F78A
:1011B000CCEFCA950000000000000000D1F716F047
:1011C0006894E9CFDA95E89431F70A9519F74CC09D
:1011D0000350033008F005E0909381008093850070
:1011E00070938400D4E6C3EFCA95000000000000AD
:1011F0000000D1F7CFEFCA95000000000000D9F73A
:10120000CCEFCA950000000000000000D1F716F0F6
:101210006894E9CFDA95E89431F70A9519F724C074
:101220009093810080938500709384000AE0D4E657
:10123000C3EFCA950000000000000000D1F7CFEF17
:10124000CA95000000000000D9F7CCEFCA95000055
:10125000000000000000D1F716F06894E9CFDA959D
:10126000E89431F70A9519F7709184008091850010
:10127000002700938100B09908C0C9E5D4E08883B5
:101280000E946002DF91CF910895DF91CF910EE02F
:101290000093B9045DDCD3E0CFEFF501CE1BDF0B8B
:1012A000F1E0EFEFEC17FD0724F4E0E2FBE1C0D83A
:1012B0000895E6E4FBE1BCD86FEF7A2D01D97B2DD0
:1012C000FFD8D3E0CFEFF1E0EFEF0881F999FECF3F
:1012D000F2BDE1BD00BDFA9AF99AD13011F4C030E7
:1012E00049F031970F93E03000E0F0070F9111F0D3
:1012F0002197EBCF0895EEE6FBE19AD82FDBD3E000
:10130000CFEFEFEFF1E0F999FECFF2BDE1BDF89A32
:1013100000B50883D13011F4C03019F0319721970E
:10132000F2CF6DEFD8D8B72EF72FD5D8A72EE72F4D
:101330000F93EF3F03E0F0070F9131F4E8E5FBE195
:101340000E9418020E94AE04089583D8C4D8172FB3
:1013500088940BD008957DD8BED8172F089405D057
:10136000089527D0712FACD808950AB1077E0AB925
:101370000BB108610BB999E04B9BFECF5C9A549876
:1013800010F05C98549A5B98539A2FD053985B9ABC
:101390002CD04B99F8CF18F05C9A549802C05C9806
:1013A000549A4B9BFECF54985C9A111F9A9521F743
:1013B00008950AB1077E0AB90BB108610BB999E02B
:1013C0004B99FECF88944C9B06C008945B98539A27
:1013D0004C99FECF04C05B98539A4C9BFECF539818
:1013E0005B9A111F9A9561F7089530E540E54A959B
:1013F000F1F73A95D9F70895CF93DF9377270E94B5
:1014000060020E9429020E946B020717D2F070FD51
:101410000BC0C7D0CFEBD4E00993099308835C9A43
:101420005498DF91CF910895C7E5D4E039D00027D3
:101430000093C204549A5C9894D0DF91CF91789431
:1014400008950CE00093B90483DB9F939FB79F93AB
:101450008F937F93EF93FF93FEE3E091C20470912B
:10146000BF048091C0049091C104E70EF81EE91FEB
:101470007491E093C20470FF0AC000005C9AFF916F
:10148000EF917F918F919F919FBF9F9118955C984D
:10149000FF91EF917F918F919F919FBF9F911895A1
:1014A000C7E5D4E03327442755279927882777278E
:1014B00000EF102E088001200294002041F030E05F
:1014C000731F40E0841F50E0951F0A94F6CF0990E7
:1014D00012940120002041F039E9731F49E9841F6B
:1014E00059E1951F0A94F6CF0880129401200294C6
:1014F000002041F03CE5731F4FE8841F52E0951F28
:101500000A94F6CF099012940120002041F039E8A6
:10151000731F41E4841F50E0951F0A94F6CF0880A2
:10152000129401200294002041F03DE8731F46E030
:10153000841F50E0951F0A94F6CF08801294012072
:10154000002041F037EA731F40E0841F50E0951FF0
:101550000A94B1F77093BF048093C0049093C104C0
:101560000895009164000F7B00936400002707BB7F
:101570000093B2000093B0000093B1000093B30059
:101580000093B40003E60093B30002E000938000F0
:1015900001E00093B10000917000026000937000C0
:1015A0000895F894002707BB0093B0000093B100A2
:1015B0000093B2000093B4000093B3000091700058
:1015C0000D7F00937000009164000064009364003C
:1015D000089518954C495320E10253495A20ED02D1
:1015E0004E455720AE0450500B20800350500D2024
:1015F0008D0350500A20550350500F206403414F73
:10160000562000045052494E0103505258200803FE
:10161000505242205A04454D49544804501A1D2046
:10162000100350501D201903464F5220E0034E4531
:1016300058542A03501C1E20330350501E20CC0344
:1016400050501C20C60350494620D60350544F200A
:10165000E20350500420E60352554E207504454ED7
:101660004420E403414E44209A034C535220A103EA
:101670004C534C20A603504F5220AB03584F5220DE
:10168000B203434F4D20B9034E454720BE03524E8F
:101690004420660444454C41EF03474F544F3B04FC
:1016A000474F53553F045245545542045448454E04
:1016B000DC034B4559204D0441434F203F03534128
:1016C00056454B094C4F41447B095045454B460319
:1016D000504F4B454D034F444220D70749444220C9
:1016E000A70753444220B90743444220C0074F5044
:1016F0004220D30753424220AA0743424220B10767
:10170000494E4220DB0749424220C8074F4443204C
:101710000E0849444320DE0753444320F007434466
:101720004320F7074F5043200A0853424320E10764
:1017300043424320E807494E4320120849424320D0
:10174000FF074F44442018084944442015085344D7
:1017500044202B084344442032084F50442045087D
:10176000534244201C08434244202308494E44204D
:101770004908494244203A0844554D50CC04454458
:10178000554D04055644554D380544535245B1094D
:101790004453434FAB0944534445A50949434720AB
:1017A0007508494345208E0849435020A2085057E8
:1017B0004D384C08505745205E0850574F2071084F
:1017C00044445320FC09414443206D0741445220C6
:1017D000920753504D20010753504F201907535083
:1017E00043202B07535057204307535052204E0796
:1017F0005350532058075457492013065457532029
:10180000BC0654575020D50654574120370654572C
:1018100057206406545752208D0654574220E8063C
:1018200000003D3D3D3D3D3D3D3D3D3D3D3D3D3D62
:101830003D3D3D3D3D3D3D3D3D3D3D3D3D3D3D3DD8
:101840003D3D3D3D3D3D3D3D3D3D3D3D3D3D3D3DC8
:101850003D3D3D3D3D3D0A0D202020202020202003
:101860002020202020202020204174746F424153EA
:1018700049432041546D6567613136380A0D202097
:101880002020202020202020202020204275696C4C
:101890006420636F64653A2032303131303532363E
:1018A0002E31383334000A0D00002D2D2D2D2D2D15
:1018B0002D2D2D2D2D2D2D2D2D2D2D2D2D2D2D2D58
:1018C0002D2D2D2D2D2D2D2D2D2D2D2D2D2D2D2D48
:1018D0002D2D2D2D2D2D2D2D2D2D2D2D2D2D0A0D7B
:1018E0002020202020204F726967696E616C206380
:1018F0006F646520284329323030322062792052CB
:101900006963686172642043617070656C730A0D6D
:101910002020687474703A2F2F70726F6A65637438
:10192000732E63617070656C732E6F726720207008
:10193000726F6A656374734063617070656C732E57
:101940006F7267200A0D2D2D2D2D2D2D2D2D2D2D56
:101950002D2D2D2D2D2D2D2D2D2D2D2D2D2D2D2DB7
:101960002D2D2D2D2D2D2D2D2D2D2D2D2D2D2D2DA7
:101970002D2D2D2D2D2D2D2D2D2D0A0D2020204DE1
:101980003136382F3332553420706F72742C205416
:1019900057492C205350492C204444532026204999
:1019A0006E70757420436170747572650A0D202025
:1019B0002020284329323031312062792053636F4F
:1019C000747420566974616C65206B73765F7072F5
:1019D0006A40626967666F6F742E636F6D200A0DCF
:1019E0002D2D2D2D2D2D2D2D2D2D2D2D2D2D2D2D27
:1019F0002D2D2D2D2D2D2D2D2D2D2D2D2D2D2D2D17
:101A00002D2D2D2D2D2D2D2D2D2D2D2D2D2D2D2D06
:101A10002D2D2D2D0A0D2020202020416C6C2072B0
:101A2000696768747320616E642072656D656469AE
:101A3000657320657870726573736C792072657355
:101A400065727665642E0A0D20202020202020203B
:101A50002020202020204E6F7420666F7220636F3C
:101A60006D6D65726369616C207573650A0D3D3D2E
:101A70003D3D3D3D3D3D3D3D3D3D3D3D3D3D3D3D96
:101A80003D3D3D3D3D3D3D3D3D3D3D3D3D3D3D3D86
:101A90003D3D3D3D3D3D3D3D3D3D3D3D3D3D3D3D76
:101AA0003D3D0A0D00002D2D2D2D2D2D2D2D2D2DE3
:101AB0002D2D2D2D2D2D2D2D2D2D2D2D2D2D2D2D56
:101AC0002D2D2D2D2D2D2D2D2D2D2D2D2D2D2D2D46
:101AD0002D2D2D2D2D2D2D2D2D2D2D2D2D2D2D2D36
:101AE0002D2D2D2D2D2D2D2D2D2D2D2D2D2D2D2D26
:101AF0002D2D2D200A0D00005661726961626C6502
:101B00007320696E2052414D3A0A0D000000454590
:101B10005020436F6E74656E74733A0A0D000000B6
:101B20004572726F723A2050726F6772616D2074E5
:101B30006F6F206C6172676520666F72204545503B
:101B4000210A0D000000536176696E6720746F20D2
:101B50004545502E0A0D00004572726F723A2045BD
:101B6000455020657261736564210A0D00004C6F59
:101B70006164696E672066726F6D204545500A0D7D
:101B8000000050524F4752414D204D656D6F7279A4
:101B900020436F6E74656E74733A0A0D00004E65D3
:101BA000787420617661696C61626C65206C6F632A
:101BB0006174696F6E3A20000000467265652020EE
:101BC00070616765733A0000202063686172733A40
:101BD00000004572726F7220303A20556E6B6E6F46
:101BE000776E20636F6D6D616E64206F72206F7011
:101BF000657261746F722E2000004572726F7220E0
:101C0000313A20456E636F756E746572656420614C
:101C10002076616C75652074686174206973206E2C
:101C20006F74206265747765656E203020616E6424
:101C3000203235352E2000004572726F7220323A04
:101C40002050726F6772616D206D656D6F727920C3
:101C500069732066756C6C2E00004572726F72207D
:101C6000333A20456E636F756E74657265642061EA
:101C700020636861726163746572207468617420A6
:101C80006973206E6F742061207265636F676E697F
:101C90007A656420747970652E2000004572726F39
:101CA0007220343A696E7465726E616C206572726E
:101CB0006F72202D20627566666572206C696D6991
:101CC0007420657863656564656400004572726FB1
:101CD0007220353A20496E617070726F707269615E
:101CE0007465207661726961626C65206E616D65F4
:101CF00020656E636F756E74657265642E000000FA
:101D00004572726F7220363A204461746120737498
:101D100061636B2070757368206572726F72202D1D
:101D2000746F6F206D616E7920617267756D656E7D
:101D30007473206F6E206F6E65206C696E652E0067
:101D400000004572726F7220373A2044617461203E
:101D5000737461636B20706F70206572726F722E86
:101D60000A0D20202020202020202046756E63743C
:101D7000696F6E20747269656420746F2075736575
:101D800020612076616C75652074686174207761CC
:101D900073206E6F7420617661696C61626C652E70
:101DA00000004572726F7220383A204D6163686995
:101DB0006E6520737461636B206572726F720A0DB9
:101DC00020202020202020202046756E6374696F1B
:101DD0006E7320616E642F6F722063616C6C732070
:101DE0006E657374656420746F6F20646565706CD4
:101DF00079206F7220746F6F20636F6D706C6578DF
:101E000000004572726F7220393A20474F544F20BC
:101E10006F7220474F5355422064657374696E6139
:101E200074696F6E206C696E6520776173206E6FC8
:101E30007420666F756E642E00004572726F72209A
:101E4000413A20537065636966696564206269740C
:101E500020706F736974696F6E2072616E676520A0
:101E60006F6620303A372065786365656465640085
:101E700000004572726F7220423A204C696E6520F4
:101E80006E756D62657220686173206D6F7265207A
:101E90007468616E207468726565206E756D657218
:101EA000616C732000004572726F7220433A2053B8
:101EB00070656369666965642062697420706F7318
:101EC0006974696F6E2072616E6765206F6620307D
:101ED0003A31206578636565646564000000457289
:101EE000726F7220443A2053706563696669656455
:101EF0002062697420706F736974696F6E207261FB
:101F00006E6765206F6620303A33206578636565BB
:101F10006465640000004572726F7220453A204982
:101F20006E70757420436170747572652072656798
:101F30006973746572206F766572666C6F770000E6
:101F40004572726F7220463A2041726974686D65FD
:101F5000746963206F766572666C6F7700004572F6
:101F6000726F722031303A2041726974686D657405
:101F7000696320756E646572666C6F7700004572E8
:101F8000726F722031313A2044697669646520624B
:101F900079207A65726F00004572726F722031325B
:101FA0003A2054574920627573206572726F72200F
:101FB0006F6363757265640000004572726F722012
:101FC00031333A2054574920696E746572666163F3
:101FD00065206E6F7420656E61626C656400000040
:101FE0004572726F722031343A2054574920536C35
:101FF000617665207265706C6965642077697468C4
:10200000204E414B00004572726F722031353A20EC
:08201000756E75736564000034
:103E000000000000000000000000000000000000B2
:103E100000000000000000000000000000000000A2
:103E20000000000000000000000000000000000092
:103E30000000000000000000000000000000000082
:103E40000000000000000000000000000000000072
:103E50000000000000000000000000000000000062
:103E60000000000000000000000000000000000052
:103E70000000000000000000000000000000000042
:103E8000FFFFFFFFFFFFFFFFFFFFFFFFFFFFFFFF42
:103E9000FFFFFFFFFFFFFFFFFFFFFFFFFFFFFFFF32
:103EA000FFFFFFFFFFFFFFFFFFFFFFFFFFFFFFFF22
:103EB000FFFFFFFFFFFFFFFFFFFFFFFFFFFFFFFF12
:103EC000FFFFFFFFFFFFFFFFFFFFFFFFFFFFFFFF02
:103ED000FFFFFFFFFFFFFFFFFFFFFFFFFFFFFFFFF2
:103EE000FFFFFFFFFFFFFFFFFFFFFFFFFFFFFFFFE2
:103EF000FFFFFFFFFFFFFFFFFFFFFFFFFFFFFFFFD2
:00000001FF
